:0200000480007A
:10000000B72F0000938F0F8073900F3015A8130047
:100010000000130000001300000013000000130094
:100020000000130000001300000013000000130084
:100030000000130000001300000013000000010086
:10004000970200009382020C73905230814001416C
:100050008141014281420143814301448144014580
:100060008145014681460147814701488148014950
:100070008149014A814A014B814B014C814C014D20
:10008000814D014E814E014F814F971102009381A6
:10009000E1C7170502001305E54A9795030093850C
:1000A000257201461122170502001305653D9705CB
:1000B0000200938565450146C52817A50300130571
:1000C000657097B503009385A56F37B6ABAB130684
:1000D000B6BAD92817B103001301C16EEF6020032F
:1000E000860293D21200F512638802008242110147
:1000F0006F00001073002030824211017300203025
:10010000711116C0F3222034E3CC02FC82421101AB
:10011000130141F806C20AC40EC612C816CA1ACC88
:100120001ECE22D026D22AD42ED632D836DA3ADCC7
:100130003EDEC2C0C6C2CAC4CEC6D2C8D6CADACC97
:10014000DECEE2D0E6D2EAD4EED6F2D8F6DAFADCA7
:10015000FEDE73252034F32510340A8601A07310C7
:10016000153492402241B2414242D2426243F243AC
:10017000025492542255B2554256D2566257F25703
:10018000064896482649B649464AD64A664BF64B33
:10019000065C965C265DB65D465ED65E665FF65F83
:1001A0001301C1077300203010C16374B50011053D
:1001B000E5BF828000000000000000000000000099
:1001C000000000000000000000000000000000002F
:1001D000000000000000000000000000000000001F
:1001E000000000000000000000000000000000000F
:1001F000197106C00AC20EC412C616C81ACA1ECC8D
:1002000022CE26D02AD22ED432D636D83ADA3EDCC6
:1002100042DEC6C0CAC2CEC4D2C6D6C8DACADECC96
:10022000E2CEE6D0EAD2EED4F2D6F6D8FADAFEDCA6
:100230009702020083A2022823A02200F322103496
:1002400096DEEF00002B170102000321A1260241D8
:10025000F65273901234B72200009382028873A082
:10026000023082403242C2425243E24372448254DC
:100270001255A2553256C2565257E2577258864806
:100280001649A649364AC64A564BE64B764C865C1A
:10029000165DA65D365EC65E565FE65F0961730059
:1002A0002030970202009382E22923A0120023A2A9
:1002B000220023A4320023A6420023A8520023AA2E
:1002C000620023AC720023AE820023A0920223A21C
:1002D000A20223A4B20223A6C20223A8D20223AA06
:1002E000E20223ACF20223AE020323A0120523A2F2
:1002F000220523A4320523A6420523A8520523AADA
:10030000620523AC720523AE820523A0920723A2C7
:10031000A20723A4B20723A6C20723A8D20723AAB1
:10032000E20723ACF207EF40D025170102000321BA
:1003300061180241F65273901234B7220000938282
:10034000028873A0023082403242C2425243E243EA
:10035000724482541255A2553256C2565257E25731
:10036000725886481649A649364AC64A564BE64B45
:10037000764C865C165DA65D365EC65E565FE65FB1
:10038000096173002030970202009382A21B83A0B0
:10039000020003A1420083A1820003A2C20083A243
:1003A000020103A3420183A3820103A4C20183A427
:1003B000020203A5420283A5820203A6C20283A60B
:1003C000020303A7420383A7820303A8C20383A8EF
:1003D000020403A9420483A9820403AAC20483AAD3
:1003E000020503AB420583AB820503ACC20583ACB7
:1003F000020603AD420683AD820603AEC20683AE9B
:10040000020703AFC20983AF820782807370043092
:10041000197106C00AC20EC412C616C81ACA1ECC6A
:1004200022CE26D02AD22ED432D636D83ADA3EDCA4
:1004300042DEC6C0CAC2CEC4D2C6D6C8DACADECC74
:10044000E2CEE6D0EAD2EED4F2D6F6D8FADAFEDC84
:100450009702020083A2020623A0220086DEEF207C
:10046000402D170102000321E1040241F65273906E
:100470001234B72200009382028873A002308240B7
:100480003242C2425243E243724482541255A25550
:100490003256C2565257E257725886481649A649F4
:1004A000364AC64A564BE64B764C865C165DA65DD0
:1004B000365EC65E565FE65F09617300203073707A
:1004C000043001A07310453082807325403073F0F2
:1004D00043308280970700009387A7FE232EB5FE46
:1004E0002322C5FA232635F82320F5F8130505F84D
:1004F0008280411106C6EF40F005EF10700901E55A
:10050000B24041018280B24041016F2080229307B6
:1005100085007D575CC118C55CC51CC9232005003A
:1005200082802328050082805C41DCC1984798C501
:1005300098474CC38CC788C91C4185071CC1828061
:100540009041FD57130785006314F60039A83E87D4
:100550005C439443E37DD6FEDCC18CC798C54CC395
:1005600088C91C4185071CC1828018495C43EDB7CE
:10057000584114451C4914C71845544154C3D84325
:100580006314A7001845D8C32328050088437D15A8
:1005900088C382803041AE8701CE4C455841B29528
:1005A0004CC563E4E5000C414CC53E856F30101F1F
:1005B0008280411122C406C62A8426C2EF209010F0
:1005C0003C44635BF0025C5085CB9304440209A871
:1005D0003C44FD173CC43C446350F0025C5089CF5E
:1005E0002685EF20A0566DD5EF2080763C44FD1780
:1005F0003CC43C44E344F0FEFD573CC4EF20D00E25
:10060000EF20500C7C40635BF0021C4885CB9304C8
:10061000040109A87C40FD177CC07C406350F002B7
:100620001C4889CF2685EF2060526DD5EF2040729F
:100630007C40FD177CC07C40E344F0FEFD577CC04D
:100640002244B240924441016F20100A29C5411151
:1006500022C426C22A8406C6AE84EF20B0063440E7
:100660005C5C1840232C0402B387F6027D5670C0F0
:1006700018C430C4B386D740BA9736975CC058C404
:1006800091EC1C489DE3EF203006B2402244924496
:100690000545410182807370043001A013050401F7
:1006A000BD3513054402A535F9BF13050401EF203C
:1006B000E0498547E319F5FC913BF1B701E573701B
:1006C000043001A0011126CA4AC84EC606CE22CC6B
:1006D000B2892E89AA84A5C53305B502130555052F
:1006E000EF3080732A8435C1930745051CC144DC73
:1006F00023202405EF20007D34405C5C18407D56AB
:10070000B387F602232C040270C018C430C413054A
:100710000401B386D740BA9736975CC058C4C53B2E
:1007200013054402ED33EF20207C23083405228595
:10073000F2406244D2444249B249056182801305C5
:100740004005EF30606D2A8401E57370043001A02C
:1007500000C071BF01E57370043001A06375B5007E
:100760007370043001A0411122C409462E848145D2
:1007700006C6A93711C500DDB2402244410182807E
:100780007370043001A05D7186C6A2C4A6C2CAC03F
:100790004EDE52DC56DA5AD85ED632C6630A051CE3
:1007A0006382051C89476399F600585D8547630598
:1007B000F7007370043001A03689AE842A84EF20DC
:1007C000A05B11E5B24781C77370043001A0EF2030
:1007D000606F185C5C5C014B894BFD59130A040186
:1007E000930A44026365F70C63077919B247638182
:1007F000072463150B002808EF206048EF20C06E27
:10080000EF10C04FEF20006C7C406394370123222F
:1008100004043C446394370123240404EF20C06C97
:100820006C002808EF20C047631E051EEF2080697A
:10083000185C5C5C630CF70AEF20006BEF208068AB
:100840003C44634FF00039A85685EF20203019C191
:10085000EF2000503C44FD173CC43C446354F0007E
:100860005C50FDF323243405EF200068EF20806501
:100870007C40634FF00039A85285EF20202D19C12C
:10088000EF20004D7C40FD177CC07C406354F0009D
:100890001C48FDF323223405EF200065EF10006BA8
:1008A000054BEF202062185C5C5CE37FF7F2304080
:1008B0006305060C631F09120844A685EF30006E1D
:1008C0001C4434405840B6971CC463EAE70A1C5CD9
:1008D00014405850850714C41CDC5DC7130544023E
:1008E000EF20C02685476311F50AC9A8EF20C05F35
:1008F000B2455285EF204007EF20C05C3C44634F77
:10090000F00039A85685EF20602419C1EF2040443B
:100910003C44FD173CC43C446354F0005C50FDF380
:1009200023243405EF20405CEF20C0597C40634F06
:10093000F00039A85285EF20602119C1EF20404115
:100940007C40FD177CC07C406354F0001C48FDF3E4
:1009500023223405EF204059EF10405F31F17D3400
:10096000054B81B73C41E38F07E27370043001A06F
:100970007370043001A0304021E61C4085C71C5C28
:10098000585085071CDC39FBEF2000560545B64062
:10099000264496440649F259625AD25A425BB25BE7
:1009A000616182804840EF2040491C5C58502322FE
:1009B000040085071CDCE31307F279D5813CE9B715
:1009C0004844A685EF30805D3C4058441440B3074E
:1009D000F0403E9758C4637CD7025840BA975CC435
:1009E00009475C506306E902185C050718DCC9DF9B
:1009F000F5B54844A685EF30605A3C405844144051
:100A0000B307F0403E9758C4E37CD7FCF9B75C507D
:100A1000185C79DB185C7D1718DC185C050718DC9E
:100A2000A5D76DBD22857136EF104052014585B7BF
:100A3000EF20804B0145A1BF411126C2AA841305B6
:100A4000400522C406C6EF30203D2A8415CD232C54
:100A50000502FD577CC10547410558DC3CC42322F3
:100A60000400232004002324040023260400232060
:100A7000040423089404613C13054402493C814664
:100A800001468145228501332285B24022449244A9
:100A9000410182800DC5411122C426C206C64AC04A
:100AA000032945002A84EF20602C8144630CA900AF
:100AB000B2402244268502499244410182807370EB
:100AC000043001A05C448544FD175CC4F5F3814605
:100AD0000146814522854539E1BF31CDA1C90111CA
:100AE00022CC26CA4AC852C406CE4EC68947B6840E
:100AF00032892E8A2A846399F600585D8547630FF0
:100B0000F7047370043001A0C932185C5C5CAA89D8
:100B10006366F70281444E857532F2406244268551
:100B20004249D244B249224A056182803C41C5DB38
:100B30007370043001A07370043001A0304041E2B2
:100B40001C40D5CB1C5C7D5785071CDC3C4463876F
:100B5000E7083C44854485073CC475BFBD32185C3A
:100B60005C5CAA89636DF702304079DA4844D2852B
:100B7000EF30C0423C4058441440B307F0403E9729
:100B800058C46375D7005840BA975CC48947E39B43
:100B9000F4FA1C5CC5DB1C5CFD171CDC65B730403F
:100BA00045D24844D285EF30603F3C405844144021
:100BB000B307F0403E9758C4E367D7FCD9BFDDF4D4
:100BC0000844D285EF30803D1C4434405840B697ED
:100BD0001CC4E3E9E7F61C401CC4ADB75C50854477
:100BE0009DDB13054402EF10707615D5E30509F27D
:100BF000232099000DB74840EF2020242322040031
:100C000091B721CD3C4181C77370043001A01C41D4
:100C1000A1CB011122CC26CA2A844AC84EC606CED0
:100C20002E896530185C5C5CAA898144637DF7007D
:100C30001C5C7D5785071CDC3C446388E7023C4410
:100C4000854485073CC44E85B538F240624426850C
:100C50004249D244B249056182807370043001A0D8
:100C60005C41C5DB7370043001A05C5099E385449E
:100C7000D9BF13054402EF10706D75D9E30909FE61
:100C800085472320F900E5B7397106DE22DC26DA34
:100C90004AD84ED652D456D232C66302051C638A55
:100CA000051AB68AAE892A84EF20000D11E5B247F5
:100CB00081C77370043001A0EF20C0201C5C6392D8
:100CC0000714B247638E070A2808EF10507BFD54C3
:100CD00013094402130A0401EF200021EF1000025F
:100CE000EF20401E7C4063949700232204043C4480
:100CF0006394970023240404EF20001F6C0028084D
:100D0000EF10107A63130518EF20C01B1C5CADCFE9
:100D1000EF20801DEF20001B3C44634FF00039A8FA
:100D20004A85EF10B06219C1EF2080023C44FD17E4
:100D30003CC43C446354F0005C50FDF324C4EF20F9
:100D4000A01AEF2020187C40634FF00039A852858C
:100D5000EF10D05F19C1EF10B07F7C40FD177CC051
:100D60007C406354F0001C48FDF364C0EF20C017C2
:100D7000EF10C01DEF2000151C5CC1E7B247A9FFB2
:100D8000EF208016014555A0EF2000161C40DDC75E
:100D9000B2454A85EF10503DEF20C0123C44634FEE
:100DA000F00039A84A85EF10705A19C1EF10507A37
:100DB0003C44FD173CC43C446354F0005C50FDF3DC
:100DC00024C4EF206012EF20E00F7C40634FF0005E
:100DD00039A85285EF10905719C1EF1070777C40F9
:100DE000FD177CC07C406354F0001C48FDF364C0D8
:100DF000EF20800FEF10801531C9EF20A00C1C5C94
:100E0000B5DFCE8522854444EFF0CFF8639C0A0419
:100E10001C5C1840FD171CDC01E7EF20601148C086
:100E20001C48A1EFEF20400C0545F2506254D2540B
:100E30004259B259225A925A21618280EF20800889
:100E40004840EF107075EF20200A99B7EFF00FDCE3
:100E50006DB73C41E38707E47370043001A0737001
:100E6000043001A05C5044C4D5DF13054402EF10E8
:100E7000F04D4DD9EFF08FD975B713050401EF1080
:100E8000F04C8547E310F5FAF5B72285EFF06FF2E5
:100E9000EF10C00B014551BF1DC9411122C44AC00A
:100EA00006C626C244412E892A84EF10306C638323
:100EB000A40281464A8681452285F933854763002D
:100EC000F502B2402244924402494101828073708B
:100ED000043001A05C44054585075CC4DDB75C4473
:100EE00085075CC4F9BF15CDADC9011122CC26CA56
:100EF0004AC84EC652C42A8406CE3289AE89EFF063
:100F0000CFDC1C5C2A8A814485E35285EFF08FDBBD
:100F1000F240624426854249D244B249224A0561E0
:100F200082807370043001A0304001CE4C445C409C
:100F3000B2954CC463E4F5000C404CC44E85EF30D0
:100F4000E0051C5C7D57FD171CDC7C40638CE700D2
:100F50007C40854485077CC04DBF3C41D9D7737028
:100F6000043001A01C4899E3854445B713050401EA
:100F7000EF10D03D75D9E30909FE85472320F9001C
:100F8000E5B721C93C41A1CDA1CB011122CC26CA94
:100F90004AC852C42A8406CE4EC62E8AEFF0EFD23B
:100FA0001C5C2A89814491CB8329C400D285228587
:100FB000EFF04FDE8544232634014A85EFF08FD0D1
:100FC000F240624426854249D244B249224A056130
:100FD00082807370043001A07370043001A0EDDFD3
:100FE0007370043001A001E57370043001A0411159
:100FF00022C42A8406C6EF10F06C005CEF10D06E9D
:10100000B240228522444101828001E573700430A0
:1010100001A0411106C622C42A84EF10B06A1C5CEC
:10102000405C1D8CEF10506C2285B240224441017F
:10103000828019C1085D82807370043001A01DCDCB
:101040009787030093870774D843630CE502D8475A
:10105000630CE504D84B6307E504D84F6302E5044D
:10106000D853630DE502D8576308E502D85B6303E4
:10107000E502D85F630EE5006F20306C73700430BA
:1010800001A001470E07BA9723A007006F20F06A5E
:101090001D47CDBF1947FDB71547EDB71147DDB760
:1010A0000D47CDB70947F9BF0547E9BF68458280BD
:1010B0006CC5828003450505828009C5085D13352E
:1010C000150082807370043001A019C51C5D485D55
:1010D0001D8D1335150082807370043001A0978731
:1010E00003009387276A984305C3984705C7984B21
:1010F00005C7984F05C7985305C7985705C7985B0C
:1011000015C7985F15C3828001470E07BA978CC335
:10111000C8C382800547D5BF0947C5BF0D47F5B78E
:101120001147E5B71547D5B71D47C5B71947F1BFF3
:101130009787030093870765D8436308E502D8477C
:10114000630BE502D84B630AE502D84F6309E50259
:10115000D8536308E502D8576307E502D85B6308F4
:10116000E502D85F6303A702828001470E07BA97A2
:1011700023A0070082800547D5BF0947C5BF0D479B
:10118000F5B71147E5B71547D5B71D47C5B7194797
:10119000F1BF411122C426C24AC02A8406C6AE84C9
:1011A0003289EF1030527840FD576314F700232244
:1011B00004043844FD576314F70023240404EF109B
:1011C000B0521C5C99E74A86A68513054402EF10CD
:1011D000B00CEF10304F3C44635BF0025C5085CBA9
:1011E0009304440209A83C44FD173CC43C446350AA
:1011F000F0025C5089CF2685EF1050156DD5EF10A9
:1012000030353C44FD173CC43C44E344F0FEFD57FC
:101210003CC4EF10704DEF10F04A7C40635BF0026D
:101220001C4885CB9304040109A87C40FD177CC0B1
:101230007C406350F0021C4889CF2685EF101011C6
:101240006DD5EF10F0307C40FD177CC07C40E3444E
:10125000F0FEFD577CC02244B24092440249410155
:101260006F10904805C579714ECE52CC06D63E8A95
:1012700022D426D24AD056CA5AC85EC662C4A547EE
:10128000BA8963F8E7007370043001A0737004300A
:1012900001A0AA8AAE843289B68B428B63090822E8
:1012A00013050006EF2050372A84630D05200A0934
:1012B000232865034A869305500A5A85EF20105C5F
:1012C00003C704001C587119230AE40203C7040071
:1012D0003E991379C9FF79C783C71400A30AF402A2
:1012E00083C71400E1C383C72400230BF40283C720
:1012F0002400CDCB83C73400A30BF40283C7340092
:10130000D5C383C74400230CF40283C74400D9CB60
:1013100083C75400A30CF40283C75400C1C783C71A
:101320006400230DF40283C76400ADCF83C774004B
:10133000A30DF40283C77400B5C783C78400230ECE
:10134000F40283C78400B9CF83C79400A30EF402CC
:1013500083C79400A1CB83C7A400230FF40283C7E3
:10136000A400A9C383C7B400A30FF40283C7B400C9
:1013700095CB83C7C4002300F40483C7C4009DC376
:1013800083C7D400A300F40483C7D40081CF83C7EC
:10139000E4002301F40483C7E40089C783C7F40091
:1013A000A301F404130B44005A85A301040423266B
:1013B000340323283405232A0404EFF08F96130501
:1013C0008401EFF00F96A947B3873741232C04041B
:1013D00000C81CCC40D023220404232E04045E86C3
:1013E000D6854A85EFF00F8F08C063040A002320DA
:1013F0008A007370043017F901001309E909832783
:10140000090097F401009384E40A91C798409C4036
:101410007C4385077CC317F701001307A7081C430B
:10142000850797F6010023AFF6069C40D5CB8327AE
:10143000090017FA0100130AAA1889EB9C40DC572F
:1014400063E6F90097F7010023A6870697F70100E6
:1014500093878703984397F60100938626045C548C
:101460009442050717F601002320E60238C463F60C
:10147000F60017F701002323F7025147B387E7026D
:10148000DA853305FA00EFF02F8A8327090081C738
:101490009C40FC43BDE383270900054499C79C4059
:1014A000DC5763F43701EFE07FF62285B250225417
:1014B00092540259F249624AD24A424BB24B224CF0
:1014C000456182805A85EF2050277D54F9BF13155E
:1014D0002600EF2070142A8BE31405DC7D54F1B74D
:1014E00097F7010023A887FC184385476301F7029B
:1014F00017FA0100130ACA0C91BF984094407C432C
:10150000FD177CC3FC42C1FB7360043069B7814A9C
:1015100017FA0100130ACA0A514CA94B33858A03F2
:10152000850A5295EFE0BFFEE39A7AFF97FB010030
:10153000938B8B155E85EFE09FFD97FA0100938AF0
:10154000EA155685EFE0BFFC17F5010013054516B7
:10155000EFE0FFFB17F501001305C516EFE03FFBB9
:1015600017F5010013054517EFE07FFA97F7010023
:1015700023A077F597F7010023AA57F3C1BD4111C6
:1015800022C406C626C24AC02A847370043097F467
:101590000100938464F09C40F9E311E497F70100A3
:1015A000938747F18043130944004A85EFE05FFCCD
:1015B0001C5489C713058401EFE09FFBCA8517F50A
:1015C000010013052510EFE03FF697F70100938720
:1015D000A7ED984397F70100938707EB9C43050716
:1015E00097F6010023A2E6EC9840850797F60100E4
:1015F00023ACF6E801CB97F701009387A7EB98435C
:10160000784349EF9C40B1C797F70100938787EA79
:101610009843630F870873700430984039EB17F7CD
:1016200001001307E7E814439442A5E27D5797F6BB
:10163000010023A9E6E4984009CF9843784311CBF1
:10164000984394437C43FD177CC3FC4299E3736049
:101650000430B2402244924402494101828097F70B
:101660000100938727E598439C437C4385077CC30F
:101670002DB794439843F8420507F8C217F70100C5
:10168000130707E314439442D5D2184358475847E9
:10169000584397F6010023A7E6DE71BF98439443B1
:1016A0007C43FD177CC3FC42B1FF7360043099BFDB
:1016B00097F701009387C7DC9C4381C773700430A0
:1016C00001A02244B2409244024941016FE01FD47C
:1016D00041C517F701001307E7DD14438147638B0A
:1016E000A606411106C622C426C27370043097F6BE
:1016F0000100938666DA9C4291C710431C437C42EA
:1017000085077CC29C42AA84404981C71C43FC4394
:10171000B9E797F701009387A7D99C43638B8704A8
:1017200097F70100938787D89C436384870497F7D2
:101730000100938767FA6309F40297F70100938722
:1017400067F86301F4028547B240224492443E8523
:10175000410182803E8582807370043001A0EF4099
:10176000701045BF9147CDB79C5493B717008907B8
:10177000E1BF8947D1BF7370043097F701009387A9
:10178000A7D1984309EF15C59C43485581CB97F7DE
:101790000100938727D29843784315E3828017F797
:1017A0000100130727D114431843F8420507F8C274
:1017B00061FD17F701001307E7CF0843F1B798431E
:1017C00094437C43FD177CC3FC42E9FB7360043007
:1017D0008280411122C42A8406C6EFE01FCF11E4A3
:1017E00097F70100938707CD80434054EFE09FCDEA
:1017F000B2402285224441018280A54763F5B700AB
:101800007370043001A0011122CC06CE26CA4AC84A
:101810004EC652C42A847370043017F901001309AC
:10182000A9C783270900D5EF79C43C486389F50827
:1018300017F70100130707C863FCB7001443638D53
:10184000860C18434457B3B4950093C4140029A0E0
:101850000443818C93B4140058546384E70A1C4CED
:101860002CC863C60700A947B385B7400CCC9317B3
:101870002700BA97584897F90100938969D48A07D5
:10188000CE97631BF702130A44005285EFE05FCE48
:1018900017F70100130787C05C5418436376F700FD
:1018A00017F70100232CF7BE5147B387E702D28513
:1018B0003385F900EFE05FC799C0EFE03FB58327BC
:1018C000090081CB97F701009387C7BE9C43FC4377
:1018D0009DEBF2406244D2444249B249224A05613A
:1018E000828097F701009387E7BC98439C437C4331
:1018F00085077CC31DF897F701009387A7BB80433A
:101900002DB74CD4A9BF6244F240D2444249B249F7
:10191000224A05616F40007581443DBF25C1011118
:1019200026CA97F401009384E4B89C4006CE22CCEA
:101930004AC84EC6638DA7027370043017F90100C0
:10194000130989B58327090091C798409C407C43BF
:1019500085077CC3584997F701009387E7D763024F
:10196000F7028327090081C79C40FC43A5EBF240A6
:101970006244D2444249B2490561828073700430A6
:1019800001A01C5517F70100130787D2E38BE7FC72
:10199000E9FB930945002A844E85EFE07FBD17F7E8
:1019A00001001307A7AF5C5418436376F70017F7DD
:1019B00001002325F7AE5147B387E70217F5010071
:1019C000130505C0CE853E95EFE01FB69C405854E8
:1019D000DC57E368F7F8EFE07FA361B76244F240B9
:1019E000D2444249B24905616F40C06715CD01112B
:1019F00022CC26CA4AC82A8406CE4EC6EFE0FFACE7
:101A0000584897F70100938727CD2A8981446300BE
:101A1000F7024A85EFE01FABF24062442685424957
:101A2000D244B249056182807370043001A01C5415
:101A300017F501001305C5C7E38DA7FCF9FB97F760
:101A400001009387E7A39C43A9EB97F701009387D5
:101A500067A69C43445493094400DC574E85B3B4B5
:101A6000F400EFE0FFB017F70100130727A35C5461
:101A7000184393C414006376F70017F70100232F6F
:101A8000F7A05147B387E70217F50100130545B3E7
:101A9000CE853E95EFE05FA9ADBF93058401EFE0F1
:101AA000BFA885BF0111056506CE22CC26CA4AC84B
:101AB0004EC652C456C25AC0EF200036630E051AF5
:101AC000AA8413050006EF2020352A84630A051C2A
:101AD00005669305500A04D92685EF20205A04583C
:101AE0008567F117BE94B7474C4593879744130A0F
:101AF00044005CD85285230C0402A301040423266D
:101B0000040223280404232A0404EFE09FA1130500
:101B10008401EFE01FA1A947232C0404F19800C819
:101B20001CCC40D023220404232E04040146971524
:101B300000009385E5B12685EFE0DF9908C073705A
:101B4000043017F90100130929958327090097F438
:101B500001009384249691C798409C407C4385075C
:101B60007CC317F701001307E7931C43850797F61B
:101B7000010023A9F6929C40C9C38327090097F965
:101B800001009389E9A381EB9C40DC5789E797F733
:101B9000010023A1879297F701009387E78E98436E
:101BA00097F601009386868F5C549442050717F6DA
:101BB0000100232BE68C38C463F6F60017F701000A
:101BC000232EF78C139527003E950A05D2854E9556
:101BD000EFE09F958327090081C79C40FC43DDE728
:101BE0008327090091C39C40EF1070498547630526
:101BF000F50C59E17370043001A097F7010023AB95
:101C0000878A1843854797F901009389699BE314F4
:101C1000F7F8CE8A17FB0100130B0BA75685D10AE4
:101C2000EFE0FF8EE31C5BFF17F501001305C5A570
:101C3000EFE0FF8D97FA0100938A4AA65685EFE000
:101C40001F8D17F501001305A5A6EFE05F8C17F5B2
:101C50000100130525A7EFE09F8B17F50100130581
:101C6000A5A7EFE0DF8A97F7010023A3678597F721
:101C7000010023AD578305B7F2406244D244424984
:101C8000B249224A924A024B0561828098409440B0
:101C90007C43FD177CC3FC42A1F77360043089B715
:101CA0006244F2404249B249224A924A024B268596
:101CB000D24405616F20602873700430FD5717E728
:101CC00001002321F77C624497E7010023A6A77C4B
:101CD000F240D2444249B249224A924A024B97E723
:101CE000010023AF077A05616FE0AFDB737004304A
:101CF00097E7010023A2077A6FE0EFE817E70100FA
:101D0000130707781C4385071CC382807370043057
:101D100097E7010093874778984305E317E70100A9
:101D20001307077808439C4381CB97E7010093870B
:101D300067789843784301EF828017E70100130723
:101D4000677714431843F8420507F8C2C1BF9843A8
:101D500094437C43FD177CC3FC42F9FF736004305D
:101D60008280411106C622C4EFE02FF697E70100FA
:101D7000938707738043EFE0EFF4B240228522445B
:101D80004101828097E701009387C7718843828071
:101D9000797106D622D426D24AD04ECE52CC56CA1B
:101DA0005AC85EC697E701009387876D9C43B1EFE1
:101DB00017E701001307C76E1C43850797E601006C
:101DC00023A0F66E832A0700638F0A0697E70100B7
:101DD0009387476B9C43814463F1FA0897E90100BC
:101DE0009389097E17EA0100130ACA6C83270A0047
:101DF0008546D85793172700BA978A07BE9983A7B5
:101E0000090063FFF600854421A897E70100938746
:101E100067689C438144850717E70100232CF76618
:101E200097E701009387C7669C4391C38544B250EE
:101E30002254268502599254F249624AD24A424BB0
:101E4000B24B4561828017E40100130464661C40B4
:101E50009C43DDC37370043001A017E40100130438
:101E6000246597E901009389A97517EA0100130A0F
:101E70006A6417EB0100130B6B621C409C43B5C3F3
:101E80001C40DC4703A9C70083274900930B490086
:101E90005E8563EEFA04EFE0AFED83278902130558
:101EA000890199C3EFE0CFEC8327C90203270B0018
:101EB000DE85139527003E950A054E956376F7005B
:101EC00017E70100232CF75CEFE00FE683270A00F9
:101ED0000327C902DC57E362F7FA1C4085449C43A0
:101EE000C5F3FD5717E70100232EF75801B717E791
:101EF00001002329F758DDBD17E701001307075B31
:101F00001C40184397E6010023A4E65A17E7010096
:101F1000232EF75897E70100938747579C4385077F
:101F200017E701002324F7561C409C4399E7FD570F
:101F300017E701002328F75451BD1C40DC47DC475C
:101F4000DC4317E70100232FF75249B597E701005B
:101F500093870753984301E77370043001A0011180
:101F600006CE22CC26CA4AC84EC652C456C25AC051
:101F70007370043097E4010093840452984061EB3D
:101F800098437D1797E6010023ACE64E9C43D9EBBE
:101F900097E70100938707519C43C9C797EA01005F
:101FA000938A0A6217EA0100130A4A4F17E90100EF
:101FB00013094950854919A83385EA00EFE0CFD6C7
:101FC000832709005854DC576379F70483A70A0F65
:101FD000C1CF83A7CA0FC04713058401EFE04FD9D3
:101FE000130B44005A85EFE0AFD85C5483260A00F7
:101FF000DA85139527003E950A052A875695E3FD55
:10200000F6FA17E70100232BF748EFE0EFD183271B
:1020100009005854DC57E36BF7FA97E7010023A94E
:1020200037476DB701449C4081CB97E70100938708
:1020300067489C43FC4395E72285F2406244D244C2
:102040004249B249224A924A024B0561828017E70F
:1020500001001307274614431843F8420507F8C246
:1020600005B7EF402000C9BF17E401001304844204
:102070001C4095C31C40054999CF193B09C597E7FA
:10208000010023A727411C40FD1717E70100232368
:10209000F7401C40FDF397E701009387673F9843A3
:1020A0008547E311F7F8EFE06FB60544ADBF11CDFA
:1020B00081E57370043001A017E701001307473C66
:1020C0001C4399C77370043001A07370043001A0E1
:1020D000411122C406C614431841850617E60100C3
:1020E0002320D63A97E601009386863B9442330438
:1020F000B70000C163F7E602637FE40063FD86007A
:1021000097E701009387073B88431105EFE04FC62F
:102110002285EF30F06E1D3D01C9B24022444101DD
:102120008280E36FE4FCD9BF2244B24041016FE0FA
:10213000EFAD11C917E70100130787341C4391C79E
:102140007370043001A06FE06FAC411106C622C469
:102150001843AA87050797E6010023A3E63297E60E
:1021600001009386263517E70100130767331843EC
:1021700088423304F7001105EFE08FBF2285EF306E
:102180003068E93311E52244B24041016FE00FA805
:10219000B240224441018280411122C406C697E721
:1021A00001009387E72D9C430144850717E7010051
:1021B0002328F72C97E701009387C72E9C4363E001
:1021C000F51217EE0100130E6E4B97E20100938299
:1021D000623E01440147854F1303500A21A0311E7E
:1021E000638DC20B83278EFFBA86F5DB8327CEFF74
:1021F000DC43232EFEFE638AC70F03AFC700DC4318
:102200002A97814E232EFEFE6385C70783A8C70049
:1022100093874803232017015CC383A788042326E0
:10222000F7011CC783A7C8021CCB83A70805232C72
:1022300007005CCB03A8080383470800639067048A
:10224000C287850783C60700B3850741E38B66FE17
:102250008981C205C181231EB700850E13070702BD
:1022600063061F038327CEFFDC43232EFEFEE39F7E
:10227000C7F983274E00232EFEFE49BF8145231E4A
:10228000B700850E13070702E31E1FFD7694131790
:102290005400311EBA86E397C2F597E70100938791
:1022A000272103AE070083270E00639D070E97E7E3
:1022B00001009387A71F03AE070083270E006392D8
:1022C000071817EE0100130EAE2F83274E109DE363
:1022D00083278E116395072019C223200600BD3184
:1022E0002285B24022444101828083274E00232E62
:1022F000FEFE21B783278E1017EF0100130F0F3D4D
:10230000DC4317E701002321F73C6380E73383A216
:10231000C700DC43AA96814E17E701002326F73A4F
:10232000914F1303500A6388E70783A8C700938778
:10233000480323A01601DCC283A7880423A6F60164
:102340009CC683A7C8029CCA83A7080523AC0600C5
:10235000DCCA03A80803834708006391672AC28781
:10236000850703C70700B3850741E30B67FE93D7D3
:102370002500C207C183239EF600850E93860602C0
:102380006386122983278E10DC4317E70100232D73
:10239000F732E39CE7F983270E1117E701002325A5
:1023A000F73261B783274E00130F8E00D4432322E8
:1023B000DE006388E629B307E500D84283A2C600A1
:1023C000814E2322EE00894F1303500A6306EF0665
:1023D0008328C7001387480323A01701D8C303A786
:1023E000880423A6F70198C703A7C80298CB03A7C0
:1023F000080523AC0700D8CB03A80803034708004F
:102400006318671C4287050783460700B305074129
:10241000E38B66FE13D7250042074183239EE70026
:10242000850E93870702638D121B83264E00D842C8
:102430002322EE00E31EEFF80327CE002322EE0056
:1024400041BF83274E00130F8E00DC432322FE0082
:102450006384E71F83A2C700DC43AA96814E232230
:10246000FE00894F1303500A6306FF0683A8C700C6
:102470009387480323A01601DCC283A7880423A600
:10248000F6019CC683A7C8029CCA83A7080523AC93
:102490000600DCCA03A80803834708006396671098
:1024A000C287850703C70700B3850741E30B67FEB3
:1024B00093D72500C207C183239EF600850E93861D
:1024C0000602638B120F83274E00DC432322FE009B
:1024D000E31EFFF88327CE002322FE0041BF83279F
:1024E000CE1197EE0100938EAE1FDC4317E701007B
:1024F0002326F71E6384D71383AFC700DC4333075B
:10250000D500014397E6010023AAF61C0D4F89422E
:102510009308500A6387D707C8479307450308C342
:102520005CC33C452326E7011CC75C551CCB1C55EE
:1025300099C3232657003C49232C07005CCB032872
:1025400005038347080063951705C287850783C67F
:102550000700B3850741E38B16FF93D72500C20719
:10256000C183231EF700050313070702638AAF0226
:102570008327CE11DC4397E6010023A1F616E39DE5
:10258000D7F983274E1297E6010023A9F61469B7FD
:102590008147231EF700050313070702E39AAFFCE8
:1025A0001A94E31C06D225BB8147239EF600850EB4
:1025B00093860602E39912F117EE0100130E4E0006
:1025C00083274E10769493165400E38307D01DB3EF
:1025D0000147239EE700850E93870702E39712E5E4
:1025E00097E70100938787EC03AE07007694931674
:1025F000540083270E00E38607CCA1B58147239EB4
:10260000F600850E93860602E39E12D783278E116D
:10261000769493165400E38107CCD1B583274E12EC
:1026200017E70100232CF70AC1BD83270E1117E716
:102630000100232BF708E1B98327CE002322FE00F7
:1026400011BD8326CE002322DE00B5B3797126D2D8
:102650004AD04ECE52CC56CA5AC85EC606D622D4EE
:1026600097E901009389C9E117E90100130949F5C8
:1026700017EA0100130A4AE297EA0100938A8AE303
:1026800097EB0100938B0BE297E401009384C4E184
:10269000054B21A883A7090003244910850717E7E4
:1026A0000100232FF7DC5D3011E89C40E5F783271C
:1026B0000900E37CFBFEEFD07FD5C5BF737004300B
:1026C00083270A00B9E383270911C0471305440093
:1026D000EFD01FEA83A70B00FD1717E701002323A4
:1026E000F7DC9C40FD1717E70100232FF7DA83275B
:1026F0000A0089C783A70A00FC4385E30858EF1046
:10270000D0032285EF1070034DB703A70A0083A7FB
:102710000A007C4385077CC37DB703A70A0083A614
:102720000A007C43FD177CC3FC42E9FB7360043064
:10273000F1B797E701009387A7D49C43DDE34111EC
:1027400006C697E7010023A507D417E70100130782
:1027500067D61C43B7A6A5A59386565A9C5B8C43A7
:10276000639BD500D0436318B60094476395C600B9
:10277000DC476388D70008430C4393854503EF206B
:10278000407897E60100938666D1904217E70100F2
:10279000130707E311A89C42B9CB9C42FD1717E62B
:1027A0000100232DF6CE904293172600B2978A0798
:1027B000BA979C43EDD3904293172600B2978A07AD
:1027C000B305F700D441A107BA97D442D4C16383BB
:1027D000F602DC46B24017E70100232DF7CC410199
:1027E0008280854717E701002324F7CA828073702F
:1027F000043001A0D1473306F602D442329754C3C5
:10280000C9BF01114AC806CE22CC26CA4EC62A89A3
:102810007370043097E40100938404C89C4017E46B
:102820000100130424C9D9E7631409000329040033
:10283000930949004E85EFD0BFD38327890289C70A
:1028400013058901EFD0DFD2CE8517E5010013050E
:10285000A5E8EFD07FCD9C4081C71C40FC43ADE391
:102860001C40638B27079C409DCF737004309C40B5
:10287000C1EB97E701009387A7C39843184325EB63
:10288000FD5717E70100232FF7BE9C4089CF1C405E
:10289000FC4391CB184014407C43FD177CC3FC42A1
:1028A00099E373600430F2406244D2444249B24931
:1028B0000561828018401C407C4385077CC3ADB70E
:1028C000184014407C43FD177CC3FC42D1FB73606D
:1028D00004301C40E39927F99C40A1C397E701000D
:1028E000938707BA9C43ADCB7370043001A09C431F
:1028F000DC47DC47DC4317E701002325F7B871B755
:1029000018401C407C4385077CC397E701009387F0
:1029100027BA984318432DD7D9BF97E7010093876B
:1029200067B817E701001307A7C99C43032787115E
:10293000631DF700F240624497E7010023AC07B63D
:10294000D2444249B249056182806244F240D24495
:102950004249B2490561F1BB6244F240D244424966
:10296000B24905616FD09FAA3DC9411126C297E4C3
:102970000100938424B44AC02E898C4006C622C428
:10298000E105EFD0FFBB88401105EFD07FBEFD57BA
:10299000630AF90497E70100938787B08043984062
:1029A0009C434A9440C3636CF40497E70100938707
:1029B00027B088438C409105EFD09FB897E701007E
:1029C000938747AC9C436376F40097E7010023AB01
:1029D00087AAB24022449244024941018280737026
:1029E000043001A08C402244B2409244024917E5D1
:1029F0000100130565CE910541016FD0FFB297E745
:102A000001009387A7AA884322448C40B240924495
:102A10000249910541016FD0BFB211C997E701008A
:102A2000938707A69C4399E77370043001A07370E5
:102A3000043001A0411126C297E40100938484A7C9
:102A40009840AE878C40B7060080D58F06C622C45A
:102A50001CCFE1053284EFD03FAD88401105EFD0A7
:102A60003FB1FD57630EF40097E70100938747A33A
:102A70008843B24092442295224441016F3040582D
:102A80008C402244B240924417E501001305C5C4AE
:102A9000910541016FD05FA925CD411126C297E470
:102AA0000100938424A14AC02E898C4006C622C40A
:102AB000E1053284EFD05FA788401105EFD05FAB0E
:102AC0008547630AF40497E701009387679D804375
:102AD00098409C434A9440C3636CF40497E7010018
:102AE0009387079D88438C409105EFD07FA597E79A
:102AF0000100938727999C436376F40097E70100D0
:102B000023A28798B2402244924402494101828024
:102B10007370043001A08C402244B24092440249B8
:102B200017E50100130545BB910541016FD0DF9FFB
:102B300097E7010093878797884322448C40B240EF
:102B400092440249910541016FD09F9F411106C6F1
:102B500022C426C25C45C04735CC93048401268537
:102B6000EFD01FA197E70100938787919C43B5E7BA
:102B7000930444002685EFD0BF9F97E70100938719
:102B8000E79158549C4363F6E70097E7010023A7B9
:102B9000E79093172700BA978A0717E501001305F6
:102BA00025A2A6853E95EFD03F9897E70100938731
:102BB00067909C4358540145DC5763F8E70085470C
:102BC00017E701002326F78C0545B24022449244C2
:102BD000410182807370043001A0A68517E50100D1
:102BE000130505ADEFD05F94C9B797E70100938750
:102BF00027899C4381E77370043001A0411106C608
:102C000022C426C2B70700804045CD8F1CC12DC409
:102C1000EFD01F96930444002685EFD07F9597E769
:102C200001009387A78758549C4363F6E70097E712
:102C3000010023A5E78693172700BA978A0717E5AF
:102C400001001305E5973E95A685EFD0FF8D97E728
:102C50000100938727869C4358540145DC5763F84D
:102C6000E700854717E701002324F7820545B240B6
:102C700022449244410182807370043001A011CD3E
:102C800097E7010093878780984397E70100938730
:102C900027819C4318C15CC182807370043001A0FD
:102CA00055C1D1CD411106C622C42A8773700430A4
:102CB00097D801009388487E83A7080091CB97D7C7
:102CC00001009387277F94439C43FC428507FCC205
:102CD00017D301001303C37C9C4103260300FD5658
:102CE0000144638FD70217DE0100130E2E7A0325ED
:102CF0000E000328070054436305A80005446371D0
:102D0000D6023308D6400544637CF80003250E0044
:102D1000918F03260300B6979CC108C350C301449A
:102D200083A7080081CB97D701009387A7789C439E
:102D3000FC4381EF2285B2402244410182807370BE
:102D4000043001A07370043001A0EF30A031DDB772
:102D5000854717D70100232DF772828019C1684576
:102D600082800145828011C16CC5828097D70100A5
:102D7000938747748843828097D701009387C771F0
:102D80009C43054589CB97D701009387676F88439C
:102D9000133515000605828031CD011126CA97D45E
:102DA0000100938424719C4006CE22CC4AC84EC6B2
:102DB0005855DC576379F7021C4D63C707009C40E8
:102DC000D457A947958F1CCD93172700BA97584918
:102DD00017D901001309C97E8A07CA97630DF70046
:102DE0009C40DC575CD5F2406244D2444249B2492F
:102DF000056182808280930945002A844E85EFD048
:102E00002FF79C4017D70100130747691843DC5779
:102E10005CD46376F70017D701002321F768139578
:102E200027003E9562440A05F240D244CE854A9579
:102E3000B249424905616FD02FEF19CD411106C645
:102E400022C426C297D701009387C76680436307D1
:102E5000A4007370043001A0014582807C4881E7A2
:102E60007370043001A054543848FD177CC8638344
:102E7000E60099C70145B240224492444101828054
:102E8000930444002685EFD0AFEE3C4817D70100ED
:102E90001307C760144329471D8F5CD418CC63F611
:102EA000F60017D70100232BF75E5147B387E702DF
:102EB00017D501001305C570A6853E95EFD0CFE666
:102EC000054555BF7370043097D701009387C75CE1
:102ED0009C4391CB97D701009387C75D98439C4350
:102EE0007C4385077CC3828097D701009387C75AAC
:102EF0009C438DC397D701009387C75B9843784362
:102F000011CB984394437C43FD177CC3FC4299E367
:102F100073600430828097D701009387A75990434C
:102F200094439843A947D456084E958F1CCF82806E
:102F300097D7010093870758984309C79443F84AE5
:102F40000507F8CA8843828079714AD006D622D410
:102F500026D24ECE2A897370043097D40100938410
:102F6000A4539C4017D401001304C454BDE31C4077
:102F7000BC4F89E71C400547F8CFD1E19C4081C791
:102F80001C40FC43F1EB737004309C408DEF1C40FF
:102F9000A84F11C5630409021C4023AC07041C4060
:102FA00023AE07049C4081C71C40FC438DEBB2500C
:102FB000225492540259F2494561828018403C4F94
:102FC000FD173CCFE9BF18401C407C4385077CC3FC
:102FD0007DBF18401C407C4385077CC349BF184017
:102FE00014407C43FD177CC3FC42F1F37360043052
:102FF000B250225492540259F249456182800840ED
:103000002EC61105EFD0CFD6B245FD576380F50629
:1030100097D701009387C74883A9070018409C43AE
:10302000AE992322370163ECF90497D70100938707
:10303000274888430C409105EFD08FD097D70100E7
:10304000938747449C4363F6F90097D7010023AB6D
:103050003743EFD0AFBB1DB7184014407C43FD177A
:103060007CC3FC428DF37360043031BF0C4017D534
:103070000100130565669105EFD00FCBD9BF97D737
:1030800001009387A74288430C409105EFD04FCBB6
:10309000C9B779714AD04ECE06D622D426D252CCA8
:1030A0002E89B2897370043097D401009384C43E92
:1030B0009C4017D401001304E43FF9EF18408947FE
:1030C000784F630CF7001C401345F5FFB84F798D1E
:1030D000A8CF1C400547F8CFADE69C4081C71C40F7
:1030E000FC43F5E3737004309C40B1E7638609004C
:1030F0001C40BC4F23A0F900184085470145784F7C
:10310000630BF7001C401349F9FF0545B84F3379AD
:10311000E90023AC27051C4023AE07049C4081C76F
:103120001C40FC43C1E3B250225492540259F2496C
:10313000624A4561828018401C407C4385077CC3FD
:1031400075B7084036C61105EFD08FC2B246FD579D
:103150006385F60897D701009387873403AA070091
:1031600018409C43369A232247016363FA0897D795
:1031700001009387E73388430C409105EFD04FBCA3
:1031800097D70100938707309C436370FA0697D75F
:10319000010023A9472F91A818401C407C438507B4
:1031A0007CC329BF184014407C43FD177CC3FC42FC
:1031B000BDFB73600430B250225492540259F2495C
:1031C000624A45618280184014407C43FD177CC3ED
:1031D000FC4289FB7360043031B70C4017D5010005
:1031E0001305854F9105EFD02FB4EFD02FA2F5B581
:1031F00097D701009387872B88430C409105EFD028
:103200002FB4E5B751C1411106C622C426C24AC037
:103210007370043097D40100938404289C40B9EB68
:1032200099C23C4D9CC2B2878946704D74CD2E87A1
:103230002A846386D70663FCF6048D456387B7004E
:1032400091456395B7006300D60C38CC8547630F72
:10325000F60405449C4081CB97D7010093878725CE
:103260009C43FC43A9E32285B24022449244024994
:103270004101828097D701009387C72398439C43DD
:103280007C4385077CC369BF7370043001A0854609
:10329000E39ED7FA3C4D33E7B70038CD45BF3C4DF0
:1032A00085073CCD65B7EF20F05B75BF130944007F
:1032B0004A85EFD0EFAB17D701001307271E5C54E8
:1032C00018436376F70017D701002329F71C5147ED
:1032D000B387E70217D501001305852ECA853E95F1
:1032E000EFD08FA41C5481C77370043001A097D70E
:1032F00001009387271C9C435854DC57E3FBE7F4F9
:10330000EFD0CF90B9B70144B1B739CD011122CC7C
:1033100026CA4AC84EC652C456C206CEBA89368A92
:10332000B2842E892A84EFD04F9AAA8A63050A00B4
:103330003C4C2320FA00784C89477CCC6389F4020A
:1033400063F4970C8D466387D40091466396D4004E
:10335000630AF70A232C24058547631EF7061C54CD
:1033600099CB7370043001A07370043001A03C4C01
:1033700085073CCCD5B797D70100938767109C434E
:10338000ADEB930444002685EFD08F9E17D7010044
:103390001307C7105C5418436376F70017D7010072
:1033A000232EF70E5147B387E70217D50100130507
:1033B0002521A6853E95EFD02F9797D701009387BB
:1033C000670F9C435854DC5763F7E7006385090097
:1033D000854723A0F90005445685EFD0AF8E22859E
:1033E000F2406244D2444249B249224A924A0561BB
:1033F00082809305840117D501001305652BEFD05A
:10340000AF9265BF0144C9BF8547E397F4F43C4CD4
:1034100033E92701232C240581B74DC1011122CCAA
:1034200026CA2A844AC806CE4EC6AE84EFD0EF899B
:103430008947744C7CCC3C4C05472A8985073CCC99
:103440006395E6061C5481C77370043001A097D7BA
:1034500001009387E7029C43ADE7930944004E8542
:10346000EFD00F9117D70100130747035C5418439F
:103470006376F70017D701002322F7025147B3877D
:10348000E70217D501001305A513CE853E95EFD0B1
:10349000AF8997D701009387E7019C435854DC57C5
:1034A00063F5E70099C085479CC06244F240D2446E
:1034B000B2494A85424905616FD0CF8073700430AC
:1034C00001A09305840117D501001305651EEFD0F7
:1034D000AF85C1B7AA8729C57370043017D701001B
:1034E000130787FB14439DE2F04F8946014563159E
:1034F000D60023AE070405451C4381CB97D70100B6
:10350000938747FB9843784315E3828097D6010061
:10351000938646FA904294427442850674C2E9B793
:1035200097D70100938707F99C437DB7984394434D
:103530007C43FD177CC3FC42E9FB7360043082804E
:103540005D71A6C2CAC052DC56DA5AD85ED686C6AB
:10355000A2C44EDE62D466D26AD017D90100130924
:1035600069F617DB0100130B2BF597D40100938448
:10357000E4F497DA0100938AAAF4054AA54B83275D
:103580000900984363010712DC4783A90700EFE0B5
:10359000EFF6EFE0AFF783270B002A8C6362F50AA2
:1035A00097D7010023AAA7F001466370351B884016
:1035B000B3858941EFD0FFBDEFE05F99630105124C
:1035C0008840814601462C00EFD00FEC4DD9A24730
:1035D000E3C807FEC24983A7490189C7138549008B
:1035E000EFC01FF9EFE08FF283270B002A8C636D89
:1035F000F508A24717D70100232087EDE3E2FBFC83
:10360000B317FA0013F70721631A071613F7770C9D
:103610006318071E93F70702C5D74E85EF00F01118
:1036200045B7DC47C04783AC0700930944004E858B
:10363000EFC01FF45C50228582975C4C6384470B7B
:1036400083270900984371FF03A70A0097D601005A
:1036500023A486E797D6010023A4F6E697D70100B6
:1036600023A2E7E6EFE09F8EA1BFDC47C04703AD92
:103670000700930C44006685EFC09FEF5C502285E5
:1036800082975C4C6386470983270900984371FF42
:1036900003A70A0097D6010023A4F6E297D70100FA
:1036A00023A2E7E2B9B7EFE06FE5EFE02FE683276B
:1036B0000B002A8CE366F5F883A70A00884081494D
:1036C0009043B385894117D70100232787DF13363D
:1036D0001600EFD01FACEFE07F87E31305EEEFC0DD
:1036E000FFD2F9BD1C4CCE85E69763E9FC049C40F3
:1036F00089CF02CA66CC22CEEFF00FE8884081461F
:1037000001464C08EFD02F8805FD7370043001A0EE
:103710001C4CE685EA97636CFD049C4089CF02CA85
:103720006ACC22CEEFF04FE58840814601464C0836
:10373000EFD06F8531F97370043001A003250900C3
:103740005CC000C8EFC0DFDFE5BDEFE03F8083274E
:103750000900DC47C047930C44006685EFC05FE179
:103760005C4C638F47035C502285829791BD032593
:1037700009005CC000C8EFC0BFDC39B7B24723AC5A
:10378000F900A5CFE29723A2F90023A83901938578
:103790004900636FFC0403A50A00EFC07FDA0DB592
:1037A0001C4C00C83387F90058C0636DEC02330C21
:1037B0003C416363FC029C4089CF02CA4ECC22CEBE
:1037C000EFF08FDB8840814601464C08EFC0BFFB1D
:1037D00059F97370043001A003A50A00E685EFC013
:1037E0003FD651B703250900E685EFC07FD5A5BFB9
:1037F00003250900EFC0DFD4E1B37370043001A0EA
:10380000B24783A6890123A839013387D70023A2B1
:10381000E9006364EC04B307FC4063EBD70483A7BF
:1038200049024E85829783A7C901E39B47D983A6A6
:103830008901B2479840B69711CF02CA3ECC4ECE0E
:10384000EFF08FD38840814601464C08EFC0BFF3AC
:10385000E31805D67370043001A06374FC00E370B4
:10386000F7FC0325090093854900EFC07FCD89BB94
:1038700003A50A0093854900EFC09FCC91B3411185
:1038800022C406C626C24AC017D40100130404C3CA
:10389000EFF04FE31C4095CBEFF00FE51C409DC3CC
:1038A000814801488147094781461306004097D562
:1038B00001009385A5B0170500001305A5C8EFD03A
:1038C0007F9A39E97370043001A017D901001309F8
:1038D000E9E14A85EFC0BFC397D40100938444E275
:1038E0002685EFC0DFC20146B145114597D70100DB
:1038F00023AA27BD97D7010023A497BCEFC01FDCE4
:1039000017D70100232CA7BA11CD97D501009385B5
:1039100065AAEFD0CFFC49B7B24022449244024995
:10392000410182807370043001A0A5C9797156CA23
:10393000AA8A1305C00222D426D24AD04ECE52CC37
:1039400006D65AC85EC63A89B689328AAE84E9215B
:103950002A8405C9EFF00FD797D70100938707B6E0
:103960009C439DCFEFF04FD8130544002320540112
:1039700004CC232E44012320340323222403EFC04C
:103980005FBA2285B250225492540259F249624AD7
:10399000D24A424BB24B456182807370043001A021
:1039A00097DB0100938B8BD45E85EFC05FB617DB8E
:1039B0000100130BEBD45A85EFC07FB50146B1452A
:1039C000114597D7010023AF77AF97D7010023A9FF
:1039D00067AFEFC0BFCE17D701002321A7AE01C943
:1039E00097D501009385059DEFD06FEFA5BF73704C
:1039F000043001A039C5011122CC06CE26CA17D445
:103A000001001304A4AB832804002A8801456385C0
:103A10000802BA842EC2368732C442C6954663C5B0
:103A2000B602EFF06FB58947630BF5020840814697
:103A300001464C00EFC03FD5F2406244D2440561DC
:103A400082807370043001A04C0081463A8646851E
:103A5000EFD0AF88F2406244D244056182800840D2
:103A6000814626864C00EFC01FD2F9B719C1084124
:103A700082807370043001A001E57370043001A0EE
:103A8000411106C622C42A84EFF0CFC3484833341C
:103A9000A000EFF06FC52285B24022444101828030
:103AA00001E57370043001A0411122C42A8406C6C6
:103AB000EFF04FC10050EFF02FC3B24022852244F7
:103AC0004101828001E57370043001A0411122C4DC
:103AD00026C22E84AA8406C6EFF0CFBE80D0224430
:103AE000B240924441016FF02FC04111714522C490
:103AF00006C61D262A8411C5232005001105EFC026
:103B00001FA12285B24022444101828001CDB70726
:103B100000FFED8F81C77370043001A099E57370C9
:103B2000043001A07370043001A0011122CC4AC8F6
:103B30004EC652C456C206CE26CABA893689B28A41
:103B40002E842A8AEFF04FA311E563850900737074
:103B5000043001A0EFE08F9A83240A00B377940029
:103B60006316090295C763870A009347F4FFE58F40
:103B70002320FA00EFE08FBDF240624426854249DF
:103B8000D244B249224A924A05618280E30DF4FC94
:103B9000E38209FEB3355001E20563050900B7076A
:103BA0000004DD8D4E86C18D13054A00EFE0FFE66F
:103BB000EFE0CFB919E1EFC07F85EFF0CFB59317F4
:103BC0006500AA8963D80700B7040001FD14B3F4A7
:103BD00099005DB7EFF00FAF83290A00B377340186
:103BE000631E090089CB63880A009347F4FFB3F78B
:103BF00037012320FA00EFF02FAFF9B7E31DF4FEF1
:103C0000DDB701C9B70700FFED8F99C773700430A6
:103C100001A07370043001A0411122C42A8406C699
:103C200026C24AC02E89EFF0EFA904409345F9FF60
:103C3000B3F795001CC0EFF02FABB24022442685AD
:103C40000249924441018280411122C42A8406C65D
:103C5000EFC0BF870040EFC0FF86B24022852244FC
:103C60004101828009C9370700FFB3F7E50099C712
:103C70007370043001A07370043001A06F204040C5
:103C8000B70700FFF18F81C77370043001A001E610
:103C90007370043001A0011122CC4AC84EC652C430
:103CA00006CE26CA3689AE892A8A3284EFF0CF8CB6
:103CB00021E1630509007370043001A0EFE00F8477
:103CC00083240A00CE855285B3E49900613FB3771F
:103CD00094006307F40683240A00EFE02FA7F24064
:103CE000624426854249D244B249224A0561828013
:103CF000EFE0CF8083240A00CE855285B3E43401FF
:103D00009537B3F78400638D8702E30609FCB70596
:103D100000054A86C18D13054A00EFE01FD0EFE091
:103D2000EFA219E1EFC08FEEEFF0EF9E9317650061
:103D3000AA8463DF0700B7070001FD17FD8C45B7B4
:103D400083270A001344F4FFE18F2320FA0071B7A0
:103D5000EFF04F9783240A00B377940063978700AE
:103D60009347F4FFE58F2320FA00EFF0EF97E1B7D8
:103D7000411122C406C62A8426C2EFD03FF85C4017
:103D800085C308489304C4006316950015A008482D
:103D900063009502B7050002EFE03FE55C40E5FBFC
:103DA0002285612A2244B240924441016FE00F9A79
:103DB0007370043001A009C9370700FFB3F7E500AD
:103DC00099C77370043001A07370043001A06F2094
:103DD000202B01C9B70700FFED8F99C7737004301E
:103DE00001A07370043001A0411122C426C206C68E
:103DF0002A84AE84EFF00F8D184093C7F4FFF98F3B
:103E00001CC02244B240924441016FF0EF8D19C1B1
:103E1000084D828001458280411122C406C62A8451
:103E2000EFD0DFED97C701009387076A9C43A1EBB2
:103E3000E56717D701001307278EF11797C6010012
:103E400023AAE66817C701002324F76817D70100E3
:103E50002326F78C97C701009387476717D7010080
:103E6000232CF78A854717C701002327076617C742
:103E70000100232D076417C701002327F76419E801
:103E8000EFE0CF8CEF10600701442285B24022445E
:103E9000410182801305840093773500C1EFE56707
:103EA0001307F5FFE917E3EDE7FC97C601009386DA
:103EB00066629C4229A0984311C7BE86BA87D84340
:103EC000E36BA7FE17C7010013074760E38AE7FA11
:103ED000984341461384870098C2D843B306A7404D
:103EE0006378D6023388A7002322D800C8C383256D
:103EF000480097C601009386E65D11A0BA869842F5
:103F00005043E36DB6FE2320E80023A00601D8430A
:103F100097C701009387875F9C43998F17C701005C
:103F20002326F75EEFE08F8231DC2285B240224407
:103F300041018280719911059DB729C9411122C49F
:103F400006C62A84EFD09FDB930584FF0326C4FFB7
:103F500017C701001307075811A03E871C43D4431D
:103F6000E3EDC6FE232CF4FE0CC397C70100938734
:103F7000E75998438327C4FF2244B240BA9717C732
:103F800001002325F75841016FD05FFC828097C75D
:103F900001009387A7578843828082803367B500EA
:103FA0000D8BAA871DE79308D6FFAA982A87AE86AD
:103FB0006371150303A8060011079106232E07FF5E
:103FC000E36A17FF9347F5FFC697F19B9107BE95EC
:103FD000AA972A9663F3C70A938645001388470079
:103FE000B3B6D70033B8050133E7F50093C6160022
:103FF000134818000D8BB3E6060113371700758FB1
:10400000330EF6409386170029CF1337AE0031EBFD
:1040100013532E002E88BE8601478328080005070B
:10402000110823A016019106E36967FE1377CEFFFE
:10403000BA95BA976302EE0483C60500138717008A
:104040002380D700637AC70283C615001387270031
:10405000A380D7006372C70203C725002381E7004E
:104060008280B307F640AE97850503C7F5FF850646
:10407000238FE6FEE39AF5FE82808280B367C50057
:104080008D8BB308C500E9C36371150FB307A0405A
:104090008D8B13873700954693F5F50F13081500A0
:1040A0003383A8407D166373D70015476363E60C1E
:1040B000D5CF2300B5000547638DE700A300B50009
:1040C0000D47130825006396E70013083500230108
:1040D000B500139685004D8E13970501518F33035C
:1040E000F34093968501D98E13562300AA97014772
:1040F00094C305079107E36DC7FE1377C3FFB307AA
:10410000E8006307E3062380B70013871700637C8A
:104110001703A380B7001387270063761703238153
:10412000B7001387370063701703A381B7001387A5
:104130004700637A17012382B7001387570063741F
:104140001701A382B700828093F5F50F13978500BE
:10415000D98D139705014D8FE37715FFAA87910736
:1041600023AEE7FEE3ED17FF828082802A8895B7B1
:104170008280AA8749BF834705002A8799C705051A
:1041800083470500EDFF198D82800145828005057A
:104190008347F5FF850503C7F5FF91C7E389E7FE70
:1041A0003385E74082808147E5BFAA87850503C73D
:1041B000F5FF8507A38FE7FE75FB82808346050028
:1041C000930700026397F600050583460500E38D1B
:1041D000F6FE938756FD93F7D70F85C7AA878145CB
:1041E00085CE01458507138606FD1317250083C676
:1041F00007003A9506053295F5F699C13305A040BA
:104200008280938536FD8346150093B5150093078C
:104210001500E1FA0145D5B7014582809C41238014
:10422000A7009C4185079CC1828097C601009386A8
:10423000E62A9C42175703001307C750138617003E
:10424000BA972380A70097C5010023A9C528A947CD
:104250006308F500930700046305F60001458280BA
:1042600075DE370610F005078347F7FF2320F6F0C9
:104270009C42FD1797C5010023A2F526EDF70145E5
:1042800082804D712322911423202115232A51135A
:10429000232481132326111423248114232E311364
:1042A000232C4113232861132326711323229113F6
:1042B0002320A113232EB111AA842E8932C6130CF8
:1042C0005002A54A8347090063808703B9CB804029
:1042D00011A0A1CB2300F40080400509050480C093
:1042E00083470900E39787FF0346190093081900E5
:1042F000C686130D0002FD597D5A0148130550056D
:104300009307D6FD93F7F70F138916006363F52A19
:1043100017C70100130707CF8A07BA979C43BA97BC
:1043200082878320C1140324811483244114032928
:1043300001148329C113032A8113832A4113032BF8
:104340000113832BC112032C8112832C4112032DE4
:104350000112832DC11171618280A14C02C4854775
:1043600063D50715B2478040938B770093F68BFF98
:1043700003AB060083A94600938786003EC6668687
:1043800081465A85CE85EF1070122AC88147638511
:104390003723930D4101854B668681465A85CE852C
:1043A000EF10E05A814666862A8BAE89EF10101016
:1043B000A24723A0AD0093861B00910D63843701B3
:1043C000B68BD9BFE37E9BFF63DD4601A2872380C6
:1043D000A70180407D1A930714009CC03E84E3C867
:1043E00046FF93962B001C08BE9631A8938777054D
:1043F0002300F4008040FD1B93871B00050480C050
:10440000F116E351F0EC9C42E3E2FAFE93870703D6
:10441000C5B79C409306000332472380D7009C40D9
:1044200093064700C14C1386170090C013068007FF
:10443000A380C700804002C4BA87050480C003ABD4
:104440000700814936C625BFB24783AC0700938B6E
:10445000470063840C1C635F40199307D002631903
:10446000FD1683C70C0085C363DC09189440850CD6
:104470007D1A2380F6008040050480C083C70C00AD
:10448000E5F7635D40018040930700022300F400DC
:1044900080407D1A050480C0E31A0AFE5EC61DB581
:1044A00002C48547A94CE3CF07EBB247804093860F
:1044B000470071B703C61600CA8699B59C4093069B
:1044C00050022380D7008040050480C0E5BBC14C6A
:1044D00002C471B5B24703C61600CA8683A9070095
:1044E00091073EC6E35E0AE04E8AFD5911BD03C640
:1044F0001600130DD002CA8621B59347FAFFFD8737
:1045000003C61600337AFA00CA86DDBB03C616005E
:10451000130D0003CA86EDB383C51600930906FD8B
:10452000CA86938705FD2E86E3EEFAFA9397290053
:10453000BE9985068609AE9983C50600938909FD53
:10454000938705FD2E86E3F3FAFE69BF32479C4050
:10455000144311073AC62380D7008040050480C069
:1045600095B3854763D3070BB24793867700E19AEB
:10457000938786003EC683A946009C4263DC090AF5
:1045800094401306D002B307F0402380C600804059
:10459000B336F000B3093041050480C03E8BB389C7
:1045A000D940A94C02C4E1BB03C616000508CA865F
:1045B00081BB9C40468921B7E37D9BDD8547814BCC
:1045C0008546E3C547E131BD97CC0100938C8CDF74
:1045D000CE856685EF00907D330AAA40635C40017A
:1045E00080402300A40180407D1A050480C0E31AA6
:1045F0000AFE014A83C70C00E38207EAE3C809E622
:10460000FD197D57E394E9E6ADBDB24793864700B7
:104610009C4336C693D9F74195B76356400193073B
:10462000D002E313FDFA97CC0100938CACD9930729
:1046300080021DBD3E8BA94C02C4804089B34D71E0
:10464000232E3113B70900409387F9FF23248114E7
:1046500023229114232C4113232A511323261114AE
:10466000232021152328611323267113232481136A
:10467000232291132320A113232EB1112A8A2EC4A1
:1046800017C40100130484E5975A0300938A8A0B28
:1046900097C40100938484AC3EC69305500229451B
:1046A00013080004B70610F083470A006386B704B6
:1046B000C1C71840050A13061700569797C801008E
:1046C00023AEC8E02300F7006382A706E31E06FDC1
:1046D000175703001307070705078347F7FF23A0B2
:1046E000F6F01C40FD1717C601002329F6DEEDF792
:1046F00083470A00E39EB7FA83461A0013051A009F
:104700002A87930B00027D5B7D5C01489305500571
:10471000A5489387D6FD93F7F70F130A170063E7B1
:10472000F5348A07A6979C43A697828717570300FC
:104730001307470155F28DBF8320C1140324811450
:1047400083244114032901148329C113032A8113EB
:10475000832A4113032B0113832BC112032C8112D3
:10476000832C4112032D0112832DC11171618280AE
:10477000A14C014D854763DB0719A2479D07E19BCB
:1047800083AD070003AB4700138787003AC46686F2
:1047900081466E85DA85EF1060512AC863066D3553
:1047A000130941018549668681466E85DA85EF10D9
:1047B000001A66868146AA8D2E8BEF10204F23208B
:1047C000A90085091109E3106DFFE3FE9DFD1306A5
:1047D0000004B70610F063D189031C40138717004B
:1047E000D69797C5010023ABE5CE23807701630CF4
:1047F000C7047D1CE3C389FFB2476800A548B386A0
:10480000F9008A061C08BE962948130300043706DF
:1048100010F0E384A6E89C429305000363F4F800DB
:10482000930570051840AE9793051700569717CE5D
:1048300001002325BECA2300F7006380072B638C89
:104840006526F116F9B7175703001307A7EF0507F9
:104850008347F7FF23A0F6F01C40FD1797C5010022
:1048600023AEF5C6EDF77D1C71B71C40130600049E
:104870001387170097C5010023A2E5C6B386FA0087
:10488000930500032380B6006300C73E890797C6DF
:10489000010023A5F6C45697930680072300D7008E
:1048A00017570300130707EAB70610F0639EC70007
:1048B00005078347F7FF23A0F6F01C40FD1717C636
:1048C0000100232DF6C0EDF7A247C14C014D910721
:1048D0002247014B832D07003EC455BDA24783AC40
:1048E000070013894700638F0C3A635480219307B4
:1048F000D002639EFB2E03C70C00BA85631007200D
:1049000025AC8547A94C014DE3C907E7A2479107AC
:10491000C1B7A24783461700528703AB0700910730
:104920003EC4E3580CDE5A8C7D5BE5B3834617002A
:10493000930BD0025287F1BB9347FCFFFD87834660
:104940001700337CFC005287E9B383461700930BB2
:10495000000352877DBB03461700138B06FD528769
:10496000930706FDB286E3EEF8FA93172B00DA9769
:1049700005078607B29703460700138B07FD9307C9
:1049800006FDB286E3F3F8FE69BFA2451C40294646
:10499000984193861700D69717C501002320D5B4F8
:1049A0002380E700138945006301C72A93070004A9
:1049B0006387F6204AC4D5B1854763DF0729A2473C
:1049C00013877700619B930787003EC4032B470042
:1049D0001C43635B0B30184013060004930617005A
:1049E00097C5010023ACD5AE56979305D00223009E
:1049F000B7006388C62CB307F0403337F000330BA1
:104A00006041BE8D330BEB40A94C014D49B3834649
:104A1000170005085287F5B9834617005287D5B9A4
:104A20001C40930600041387170017C601002327B4
:104A3000E6AAD697130650022380C700E31FD7C407
:104A400017570300130707D0B70610F00507834771
:104A5000F7FF23A0F6F01C40FD1717C60100232F17
:104A6000F6A6EDF71DB9C14C014D29B31C409306C4
:104A700000042A8A1387170017C601002320E6A620
:104A8000D697130650022380C700E318D7C01757E4
:104A90000300130727CBB70610F005078347F7FF7E
:104AA00023A0F6F01C40FD1717C601002328F6A22C
:104AB000EDF72A8ADDB6175703001307A7C80507C5
:104AC0008347F7FF2320F6F01C40FD1797C5010030
:104AD00023A6F5A0EDF7F1162DBB1757030013071A
:104AE00067C6F1FDF11635B3E3FC9DCB8549C5B131
:104AF000014C03C70C00BA85E30E07EAFD582945AF
:104B000013080004B70610F063570B0A1C40138605
:104B10001700D69717C301002322C39C2380E70008
:104B20006384A50663040609850C03C70C007D1C7D
:104B3000BA8579FBE35080E91C4093050002130617
:104B40000004B70610F021A07D1CE3050CE61387D6
:104B50001700D6972380B70017C501002320E598DA
:104B6000BA87E313C7FE175703001307A7BD05074E
:104B70008347F7FF23A0F6F01C40FD1717C501007F
:104B8000232EF594EDF7C9B717570300130787BB1A
:104B900041DE05078347F7FF23A0F6F01C40FD1711
:104BA00017C60100232CF692EDF7BDBF175703007F
:104BB000130747B9F9BF7D1BE31A1BF5A5BF1757AC
:104BC0000300130727B8B70610F005078347F7FF60
:104BD00023A0F6F01C40FD1717C601002320F69015
:104BE000EDF74AC45DBC97BC0100938CAC7DDA85BF
:104BF0006685EF00B01B330CAC40E35C80EF1C40DB
:104C000013060004B70610F021A07D1CE3020CEE91
:104C100013871700D6972380770197C5010023AF2C
:104C2000E58ABA87E313C7FE17570300130787B156
:104C300005078347F7FF23A0F6F01C40FD1797C533
:104C4000010023ADF588EDF7C9B717570300130727
:104C500067AFB5FA4AC491B4A247138747009C4393
:104C60003AC413DBF741B5B317570300130787ADF9
:104C7000B70610F005078347F7FF23A0F6F01C40A6
:104C8000FD1717C60100232BF684EDF7854717C7DC
:104C900001002325F7849307800717570300230398
:104CA000F7AA1DB1635680019307D002E39DFBF282
:104CB00097BC0100938C0C7113078002930580024E
:104CC00035BD975603009386E6A7370610F0850694
:104CD00003C7F6FF2320E6F018407D1797B50100C3
:104CE00023AEE57E6DF701BBBE8DA94C014D45B4E9
:104CF000B70710F023A0A7F201A0397113034102F6
:104D00002ED29A8506CE32D436D63AD83EDA42DC56
:104D100046DE1AC62D32F2400145216182805D7166
:104D20001303810322D42AC632DC2A841A8668003F
:104D300006D6BEC236DEBAC0C2C4C6C61ACEEFF0B0
:104D40004FD4B247238007003245B250018D225420
:104D500061618280B70710F083A647F403A607F4C9
:104D600003A747F4E31AD7FE8566938606FAB29640
:104D700033B6C600B305E60023A4D7F423A6B7F4E0
:104D80008280B70710F003A747F403A607F483A6B1
:104D900047F4E31AD7FE8566938606FAB29633B6D1
:104DA000C60023A4D7F4B305E60023A6B7F49307FF
:104DB000000873A047308280411122C406C65144C6
:104DC0007D14552575FCB240224441018280411179
:104DD00022C406C697B701009387C77017B40100B5
:104DE0001304047098431C401306F07C9306470696
:104DF0009387470697B5010023A6D56E97B50100A6
:104E000023A0F56E6346D600B24022444101828061
:104E10001307478997B7010023A6E76CEF00C0721C
:104E20008547631FF500184085679387F77601452E
:104E3000E3DCE7FC753D2244B24041016FC01FEB4B
:104E400017B50100130585584D3D094555352244D8
:104E5000B24041016FC09FE917B501001305055924
:104E600069BD17B501001305E55841BD411122C4C4
:104E700026C206C6856417B401001304245893871C
:104E800084380100FD17F5FF2285EFF01FE7C5BF4D
:104E9000411106C622C4792317070000130707F241
:104EA000814605469305200317B501001305855576
:104EB000EFE0BFA72A84EFC07FE52A86228522443F
:104EC000B24001478146854541016FE0BFB24111C3
:104ED00006C69D2D054781476316E500B2403E8515
:104EE0004101828017B501001305454EEFF0FFE048
:104EF000B24089473E85410182807370043001A031
:104F000082807370043001A097B601009386865E9C
:104F10009C4237575A01130757E3B387E7028507C7
:104F2000139517009CC245818280411106C697B730
:104F300001009387275D8843814609468145EFE05C
:104F40006FACEFD03FF817B701001307275B1C4386
:104F500085071CC3B24041016FD01FF9397106DECD
:104F600022DC26DA4AD84ED652D456D25AD05ECE59
:104F700062CCEFC0BFD92A84930640063000814539
:104F80007D55EFE00F91AA84EFC05FD8018D9307A4
:104F9000300663E6A70097B7010023AD075681C42A
:104FA0007370043001A0A24781C77370043001A060
:104FB00017B40100130404550840E165740011465C
:104FC0009385156AEFE00FA485476305F5007370BC
:104FD000043001A0B249638509007370043001A058
:104FE000EFC0DFD22A8993064006300081457D5507
:104FF000EFE02F8AAA84EFC07FD1330525419307C4
:10500000300663F6A70097B7010023A50750854730
:105010006385F4007370043001A0A24AE1679387AE
:10502000176A6385FA007370043001A017BA010093
:10503000130A8A4D83270A000840814685071146D6
:10504000D68517B701002321F74CEFE0AF9B63052E
:1050500095007370043001A008400569814611462F
:105060009305395BEFE00F9A01C57370043001A01E
:105070008146300081457D55EFE0AF8163059500A5
:105080007370043001A0A24563855501737004302C
:1050900001A0084081460D46EFE0CF9663059500DC
:1050A0007370043001A0084081460D469305395BBA
:1050B000EFE04F95630595007370043001A08146C1
:1050C000300081457D55EFD0DFFC6305950073709E
:1050D000043001A0A2471309395B6385270173706F
:1050E000043001A00840E165814601469385156AB8
:1050F000EFE04F9185476305F5007370043001A020
:105100008146300081457D55EFD0BFF82247856745
:105110009387375B6305F7007370043001A09544F3
:1051200005490840814609468145EFE0AF8DFD14F1
:10513000631E2501FDF48146300081457D55EFD089
:105140005FF5630825017370043001A073700430AB
:1051500001A0224785679387875B6305F70073701B
:10516000043001A08146300081450145EFD07FF237
:1051700001C57370043001A08146300081457D5522
:10518000EFD03FF18544FD5A0840A685814605468B
:10519000EFE04F878146300081450145EFD07FEF3A
:1051A00085472A89631EF500A24785098604E39D89
:1051B00057FD930700026388F9007370043001A063
:1051C0007370043001A09306400630008945EFD08B
:1051D0005FEC01C57370043001A0084081460146B0
:1051E000FD55EFE02F828146300081450145EFD02B
:1051F0005FEA630525017370043001A0A244F957EA
:105200006385F4007370043001A0084081460146B4
:105210008145EFD03FFF8146300089450145EFD001
:105220005FE7A247638597007370043001A0814651
:10523000300081450145EFD0DFE501C573700430D2
:1052400001A0A244F1576385F4007370043001A0FB
:105250000840740005468145EFD0DFFAA247638518
:1052600097007370043001A03000FD558146014560
:10527000EFD03FE20840740005468145EFD09FF82B
:105280003249630509007370043001A09D498544CB
:105290000840A68574000546EFD0DFF6B247FD1939
:1052A00063942703336999008604E39309FE8146DA
:1052B000300081457D55EFD0DFDD0145EFE08FA166
:1052C00019C57370043001A07370043001A0084048
:1052D000E165740011469385156AEFD0BFF2014570
:1052E000EFE04F9F85476305F5007370043001A020
:1052F0000145EFE02F9E01C57370043001A08327A4
:105300000A0081460146850781457D5517B7010092
:10531000232CF71EEFD0FFD717070000130727C174
:10532000814601469305A00517B501001305C50E7A
:10533000EFE0AFDF37595A01A16497B7010023AD01
:10534000A71A97BB0100938BEB1A17BC0100130C33
:10535000AC1A97B901009389A91A130959E3FD14EE
:10536000130BA005A94A83A70B0003250C007D574A
:10537000B387270381469145850713D60701658EBC
:105380003376660317B401002326F41663735601BF
:105390002946EFE02FE683A70B000145B3872703DB
:1053A000850713D40701658C3374640317B70100B4
:1053B0002322F714637354012944A285EFD0DFB888
:1053C000814501C983A70900850717B70100232973
:1053D000F7120145EFD05FB7A28501C983A7090085
:1053E000850717B70100232DF7100545EFD0DFB56E
:1053F00083A70900FD55AA97054517B7010023218A
:10540000F710EFD07FB403A7090083270A002A977B
:10541000850797B6010023A5E60E17B701002325DF
:10542000F70E91B7411197B701009387A70D014778
:105430008148014881461306004097B501009385D5
:1054400065FE170500001305A5B106C6EFB09FE184
:10545000B24097070000938767AB17B70100232B73
:10546000F7084101828097B701009387E7089C43C2
:10547000ADC397B701009387A7079C431307100399
:1054800085076353F704011122CC06CE17B401003F
:105490001304C4051C4017B70100232B070405475C
:1054A000638FE70609476386E7048DC797B7010056
:1054B0009387C7049C43F2406244850717B70100F5
:1054C000232EF7020561828017B701002322F7021D
:1054D0008280828097B701009387C7028843814505
:1054E000EFD0BFF31C40850717B701002320F7005A
:1054F00075BF97B701009387E70088431304F00F47
:10550000014774000946814522C6EFD01FE0B2472B
:105510006389870297B7010023AA07FC41BF97B7A9
:105520000100938727FE884301478146094681454C
:10553000EFD0BFDD1C40850717B701002328F7FA1D
:10554000B5B77370043001A097B701009387C7FB0C
:1055500097B60100938646F9984394426383E60424
:105560009C4317B701002321F7F897B701009387F1
:10557000E7F817B701001307A7F89C431843637CAB
:10558000F700998F15476378F70097B7010023A3B9
:1055900007F80145828097B701009387A7F78843F2
:1055A000828097B7010023A707F6C1B7AA95AA87FB
:1055B0006385B70003C7070001E73385A7408280F2
:1055C0008507FDB7814863DA05003305A040B3378E
:1055D000A000B305B0409D8DFD5863D90600330689
:1055E000C040B337C000B306D0409D8E32883683AA
:1055F000AA872E87639F061C97B60100938686CBE9
:1056000063F1C50C416E6377C60B130EF00F637325
:10561000CE002143335E6600F29603CE06001A9E4A
:10562000130300023303C341630C0300B395650009
:10563000335EC501331866003367BE00B3176500DB
:10564000135E0801B355C70313150801418193D6B2
:1056500007013376C703B305B5024206D18E63F85E
:10566000B600C29663E5060163F3B600C2968D8E5E
:1056700033F7C603C207C183B3D6C603B306D50248
:1056800013150701C98F63F8D700C29763E50701B7
:1056900063F3D700C297958F33D567008145638A3E
:1056A0000800B307A0403337F000B305B0403E8593
:1056B000998D8280370E00014143E36DC6F5614349
:1056C00091BF01E605483358680241676373E808F3
:1056D0001307F00F63730701214333576800BA962D
:1056E00003C606001A96130300023303C34063196E
:1056F0000306B3850541935608011315080141813E
:1057000013D6070133F7D502B3D5D5024207518F1F
:10571000B305B5026378B700429763650701637309
:10572000B7004297B305B74033F7D502C207C1832C
:10573000B3D5D502B305B50213150701C98F63F8B8
:10574000B700C29763E5070163F3B700C2978D8F77
:10575000A1B7370700014143E361E8F86143B5BFF2
:105760003318680033DEC500935E08013356C50068
:10577000B31765003355DE03B39565004D8E931561
:105780000801C181935606013377DE033385A502F4
:105790004207558F6378A7004297636507016373DB
:1057A000A7004297B306A74033F7D60342064182CB
:1057B000B3D6D6034207B386D502B365C70063F8F4
:1057C000D500C29563E5050163F3D500C295958DBB
:1057D0001DB7E3E6D5EC416863F50605930EF00FBF
:1057E00033B8DE000E0833DE060117B301001303E1
:1057F00063AC7293834E0300130E0002C29E330EFD
:10580000DE4163170E0263E4B6006369C500B307A7
:10581000C540958D3335F5003387A5403E85BA8563
:10582000BDBD370300014148E3EF66FA614865BF3B
:105830003357D601B396C601D98EB357D50133D7A6
:10584000D501B395C501CD8F93D506013373B7024A
:10585000139F0601135F0F0113D807013316C6010A
:105860003315C5013357B702420333680301B30F41
:10587000EF023A83637CF80136981303F7FF6367FE
:10588000D8006375F8011303E7FF36983308F84131
:10589000B37FB8023358B802C20FB3050F03139F8A
:1058A0000701135F0F0133EFEF014287637CBF00F5
:1058B000369F1307F8FF6367DF006375BF001307A8
:1058C000E8FF369F4203C16F3363E3009387FFFF16
:1058D00013580601330FBF40B375F3001353030190
:1058E000F18F3387F502B307F302B3850503330362
:1058F0000303BE95135807012E986373F8007E9337
:10590000C167FD17935508013378F80042087D8F71
:105910009A9542976366BF00631BBF006379E500F9
:105920003306C7403337C700958D998D32873307CB
:10593000E5403335E500B305BF40898DB397D50108
:105940003357C70133E5E700B3D5C50189BBAE873F
:10595000328836872A836396062097B80100938899
:10596000689563FEC50A41676374E60A1307F00F82
:105970003337C7000E07B356E600B69883C6080053
:10598000369793060002998E99CAB397D70033577A
:10599000E5003318D600B365F7003313D50013556F
:1059A0000801B3D7A50213160801418293560301DB
:1059B00033F7A502B305F6024207D98E3E8763FC92
:1059C000B600C2961387F7FF63E7060163F5B600DA
:1059D0001387E7FFC2968D8EB3F7A60242031353D7
:1059E0000301B3D6A602C20733E36700B305D602AC
:1059F0003685637BB30042931385F6FF636603012C
:105A00006374B3001385E6FF4207498F81454DA8B3
:105A1000B70600014147E360D6F66147A9BF01E63A
:105A2000854633D8C602C166637ED8089306F00F58
:105A300063F306012147B356E800B69883C6080011
:105A4000BA9613070002158F49E7B38707418545CA
:105A5000135608019318080193D8080193560301BF
:105A600033F7C702B3D7C7024207D98E3385F8028E
:105A70003E8763FCA600C2961387F7FF63E7060123
:105A800063F5A6001387E7FFC296898EB3F7C602B7
:105A9000420313530301B3D6C602C20733E36700C0
:105AA000B388D8023685637B130142931385F6FFD2
:105AB00063660301637413011385E6FF4207498F90
:105AC0003A858280B70600014147E366D8F6614710
:105AD0009DB73318E800B3D5D7003313E500B356AC
:105AE000D50013550801B397E70033F7A502B3E8D3
:105AF000F60093170801C18313D60801B3D5A50298
:105B00004207518FB386B7022E86637CD700429737
:105B10001386F5FF636707016375D7001386E5FFFA
:105B20004297B306D74033F7A602C20893D80801BC
:105B3000B3D6A6024207B385D702B36717013687EB
:105B400063FCB700C2971387F6FF63E7070163F5AD
:105B5000B7001387E6FFC2978D8F93150601D98D85
:105B6000C5BD63E2D514416763FEE6021308F00F7A
:105B70003337D8000E0733D8E60097A50100938588
:105B80006573C29503C80500930500023A98B38572
:105B9000054185E10547E3E5F6F23335C5001347D6
:105BA000150039BFB70500014147E3E6B6FC614780
:105BB000D9B733570601B396B600D98E93DE0601E6
:105BC00033D70701B378D703B397B700335805012C
:105BD0003363F80093970601C1831358030133160A
:105BE000B6003357D703C20833E80801338FE70202
:105BF0003A8E637CE8013698130EF7FF6367D8008E
:105C00006375E801130EE7FF36983308E841B3786F
:105C1000D8033358D803C208B38E07039317030180
:105C2000C183B3E7F800428763FCD701B697130737
:105C3000F8FF63E7D70063F5D7011307E8FFB697CE
:105C4000420EB387D741C16E3367EE001388FEFF63
:105C50003373070193580701337806014182330EED
:105C600003033388080393560E013303C3024293A0
:105C70009A96B388C80263F30601F69813D6060114
:105C8000B29863E01703E39317D9C167FD17FD8E40
:105C9000C206337EFE003315B500F2968145E371EE
:105CA000D5E27D17A5B38145014719BDB288368776
:105CB000AA872E886398061C97A601009386865FA4
:105CC00063F8C50A4163637E66081303F00F6373CC
:105CD000C30021473353E6009A9603CE0600130310
:105CE00000023A9E3303C341630C0300B395650081
:105CF000335EC501B31866003368BE00B317650094
:105D000013D608013377C80213950801418193D651
:105D100007013358C8024207D98E3308050363F8D8
:105D20000601C69663E5160163F30601C696B386BF
:105D3000064133F7C602C207C183B3D6C602B30613
:105D4000D50213150701C98F63F8D700C69763E51D
:105D5000170163F3D700C697958F33D56700814548
:105D60008280370300014147E36666F661479DB7CD
:105D700001E60546B3581603416663F3C8081306E7
:105D8000F00F63731601214733D6E800B29603CEB5
:105D90000600130300023A9E3303C341631903064E
:105DA000B385154113D7080113950801418113D616
:105DB0000701B3F6E502B3D5E502C206D18EB305FD
:105DC000B50263F8B600C69663E5160163F3B60044
:105DD000C696B385B640B3F6E502C207C183B3D514
:105DE000E502B305B50213950601C98F63F8B70044
:105DF000C69763E5170163F3B700C6978D8FB1BFF0
:105E0000370600014147E3E1C8F86147B5BFB398E1
:105E1000680033D7C501B3176500335EC50113D5DC
:105E20000801B376A702B3956500336EBE00939563
:105E30000801C18113560E013357A702C206D18E45
:105E40003387E50263F8E600C69663E5160163F35F
:105E5000E600C6963386E640B376A602420E135E8F
:105E60000E013356A602C2063386C502B3E5C6014B
:105E700063F8C500C69563E5150163F3C500C695D3
:105E8000918D0DB7E3EED5EC416763F5E604930E13
:105E9000F00F33B7DE000E0733D3E60097A80100FA
:105EA000938848419A9883CE0800130E0002BA9E48
:105EB000330EDE4163170E0263E4B6006369C5006A
:105EC000B307C540958D3335F5003388A5403E8531
:105ED000C28579B5B70800014147E3EF16FB61477A
:105EE00065BF3357D601B396C601D98EB357D501D6
:105EF00033D7D501B395C501CD8F93D50601337343
:105F0000B702139F0601135F0F0193D807013316E1
:105F1000C6013315C5013357B7024203B3681301F5
:105F20003308EF023A8363FC0801B6981303F7FFC6
:105F300063E7D80063F508011303E7FFB698B38859
:105F40000841B3FFB802B3D8B802C20FB3051F03AC
:105F5000139F0701135F0F0133EFEF014687637C47
:105F6000BF00369F1387F8FF6367DF006375BF00CC
:105F70001387E8FF369F4203C1683363E3009387CA
:105F8000F8FF13580601330FBF40B375F3001353E6
:105F90000301F18F3387F502B307F302B3850503DD
:105FA00033030303BE95135807012E986373F8005B
:105FB0004693C167FD17935508013378F8004208EE
:105FC0007D8F9A9542976366BF00631BBF0063791C
:105FD000E5003306C7403337C700958D998D32876A
:105FE0003307E5403335E500B305BF40898DB397EE
:105FF000D5013357C70133E5E700B3D5C5018DB3EC
:1060000097A701009387074B944317A70100130735
:1060100027491843C8C2637BE50017A7010013078F
:10602000E74808438C4391056FA08FD1411122C4EA
:1060300006C617A701001307A7472A8408438C4305
:106040009105EFA0EFCF97A701009387A7439C434B
:106050006376F40097A7010023A68742B24022444A
:106060004101828097A701009387C74498439443D6
:106070007C43FD177CC3FC4299E37360043082804B
:10608000011122CC26CA2A84AE844AC84EC652C404
:1060900056C206CEEFB09FC61C4003290401B709C3
:1060A0000001B3E59700930AC4000CC08144FD19B8
:1060B000370A00021840638C2A03032609004A8528
:1060C000B3654701B376360193175600758F0329E0
:1060D000490063C4070001E7F1BFE39DE6FC9317A5
:1060E000760063D30700D58CEFC03FB0E1B793C40F
:1060F000F4FFF98C04C0EFB07FE50840F240624441
:10610000D2444249B249224A924A056182804111F1
:1061100006C622C4EFE0DFD717F7FFFF130767CBF0
:10612000814605469305400617A501001305052E77
:10613000EFD0AFFF19C92A84EFB05FBD2A860147AF
:10614000814685452285EFD0FF8AEFB0BF95B240EA
:08615000224401454101828057
:02000004800278
:10000000B444FEFFB245FEFFBC44FEFFB245FEFF16
:10001000B245FEFFB245FEFFB245FEFFD444FEFFEF
:10002000B245FEFFB245FEFFEE44FEFFFA44FEFF7E
:10003000B245FEFF0C45FEFF1845FEFF1845FEFFCA
:100040001845FEFF1845FEFF1845FEFF1845FEFF48
:100050001845FEFF1845FEFF1845FEFFB245FEFF9E
:10006000B245FEFFB245FEFFB245FEFFB245FEFFC0
:10007000B245FEFFB245FEFFB245FEFFB245FEFFB0
:10008000B245FEFFB245FEFFB245FEFFB245FEFFA0
:10009000B245FEFFB245FEFFB245FEFFB245FEFF90
:1000A000B245FEFFB245FEFFB245FEFFB245FEFF80
:1000B000B245FEFFB245FEFFB245FEFFB245FEFF70
:1000C000B245FEFFB245FEFFB245FEFFB245FEFF60
:1000D000B245FEFFB245FEFFB245FEFFB245FEFF50
:1000E000B245FEFFB245FEFFB245FEFFB245FEFF40
:1000F000B245FEFFB245FEFFB245FEFFB245FEFF30
:100100004C45FEFF6245FEFFB245FEFFB245FEFFD5
:10011000B245FEFFB245FEFFB245FEFFB245FEFF0F
:10012000B245FEFFA845FEFFB245FEFFB245FEFF09
:100130005A43FEFF1244FEFFB245FEFFB245FEFFEA
:100140004844FEFFB245FEFFA044FEFFB245FEFF5D
:10015000B245FEFFCE44FEFFC048FEFF1449FEFF3D
:10016000C848FEFF1449FEFF1449FEFF1449FEFF74
:100170001449FEFFBA47FEFF1449FEFF1449FEFF73
:10018000D447FEFFE047FEFF1449FEFFF247FEFFA3
:10019000FE47FEFFFE47FEFFFE47FEFFFE47FEFF57
:1001A000FE47FEFFFE47FEFFFE47FEFFFE47FEFF47
:1001B000FE47FEFF1449FEFF1449FEFF1449FEFFEF
:1001C0001449FEFF1449FEFF1449FEFF1449FEFFC7
:1001D0001449FEFF1449FEFF1449FEFF1449FEFFB7
:1001E0001449FEFF1449FEFF1449FEFF1449FEFFA7
:1001F0001449FEFF1449FEFF1449FEFF1449FEFF97
:100200001449FEFF1449FEFF1449FEFF1449FEFF86
:100210001449FEFF1449FEFF1449FEFF1449FEFF76
:100220001449FEFF1449FEFF1449FEFF1449FEFF66
:100230001449FEFF1449FEFF1449FEFF1449FEFF56
:100240001449FEFF1449FEFF1449FEFF1449FEFF46
:100250001449FEFF1449FEFF3248FEFF6048FEFFCE
:100260001449FEFF1449FEFF1449FEFF1449FEFF26
:100270001449FEFF1449FEFF1449FEFFB648FEFF75
:100280001449FEFF1449FEFF1846FEFF1247FEFF09
:100290001449FEFF1449FEFF8447FEFF1449FEFF88
:1002A000AA47FEFF1449FEFF1449FEFF0E49FEFF58
:1002B000000102020303030304040404040404040D
:1002C00005050505050505050505050505050505DE
:1002D00006060606060606060606060606060606BE
:1002E00006060606060606060606060606060606AE
:1002F000070707070707070707070707070707078E
:10030000070707070707070707070707070707077D
:10031000070707070707070707070707070707076D
:10032000070707070707070707070707070707075D
:10033000080808080808080808080808080808083D
:10034000080808080808080808080808080808082D
:10035000080808080808080808080808080808081D
:10036000080808080808080808080808080808080D
:1003700008080808080808080808080808080808FD
:1003800008080808080808080808080808080808ED
:1003900008080808080808080808080808080808DD
:1003A00008080808080808080808080808080808CD
:1003B000546D725100000000546D7220537663003A
:1003C000286E756C6C2900004572726F7220696E20
:1003D000205461736B4E6F74696679207461736B1E
:1003E00073200D0A000000006D69616F750A00003E
:1003F0006D69616F75320A0068756E6772790A00FF
:1004000054696D6572320000436865636B54696DB1
:10041000657200004E6F74696669657200000000C5
:0C0420004E6F746966696564000000009E
:10042C001000000000000000017A5200017C010164
:10043C001B0D020010000000180000007C51FEFF94
:10044C008A03000000000000100000002C000000D7
:10045C00F254FEFF5E0300000000000010000000DC
:10046C00400000003C58FEFF540300000000000058
:0C050800FC8F0100090000000100000051
:040000058000004037
:00000001FF
